:0200000480007A
:100000006F008004732F2034930F80006308FF0378
:10001000930F90006304FF03930FB0006300FF038E
:10002000130F000063040F0067000F00732F2034CC
:1000300063540F006F00400093E19153171F0000BD
:1000400023223FFC6FF09FFF93000000130100008C
:10005000930100001302000093020000130300004C
:100060009303000013040000930400001305000034
:10007000930500001306000093060000130700001C
:100080009307000013080000930800001309000004
:1000900093090000130A0000930A0000130B0000EC
:1000A000930B0000130C0000930C0000130D0000D4
:1000B000930D0000130E0000930E0000130F0000BC
:1000C000930F0000732540F16310050097020000B4
:1000D000938202017390523073500018970200000F
:1000E00093824202739052309B021000939252030B
:1000F0009382F2FF7390023B9302F0017390023AF5
:100100007350403097020000938242017390523046
:10011000735020307350303093010000970200007C
:10012000938282EE73905230130510001315F5017F
:10013000635C05000F00F00F930110009308D005D9
:10014000130500007300000093020000638A0200A0
:1001500073905210B7B200009B82921073902230BD
:100160007350003097020000938242017390123462
:10017000732540F1730020309301200093000000AC
:100180001301000063F620006314303E6316300054
:10019000E3FE20FE631E303C93013000930010000C
:1001A0001301100063F620006314303C6316300026
:1001B000E3FE20FE631E303A930140009B001000D6
:1001C000939000029380F0FF1B01100013110102B5
:1001D0001301F1FF63F62000631C30386316300012
:1001E000E3FE20FE631630389301500093001000A8
:1001F0001301000063F62000631C303663163000E4
:10020000E3FE20FE63163036930160009B00100071
:10021000939000029380F0FF1B0110001311010264
:100220001301E1FF63F620006314303463163000DD
:10023000E3FE20FE631E3032930170009B0010002D
:10024000939000029380F0FF1301000063F62000FA
:100250006310303263163000E3FE20FE631A303044
:1002600093018000930000001301100063F420004C
:1002700063143000631E302EE3FE20FE93019000D5
:100280009B001000939000029380E0FF1B01100080
:10029000131101021301F1FF63F420006314300015
:1002A0006318302CE3FE20FE9301A00093000000B1
:1002B0001B011000131101021301F1FF63F4200070
:1002C000631430006316302AE3FE20FE9301B00071
:1002D000B70000809B80F0FF1B0110001311F1019B
:1002E00063F420006314300063143028E3FE20FE22
:1002F0009301C000130200009B00F0009390C00126
:100300009380F0FF1B01F0001311C10163F220265E
:100310001302120093022000E31052FE9301D0005A
:10032000130200009B00F0009390C0019380F0FF47
:100330001B01F0001311C1011300000063FA202219
:100340001302120093022000E31E52FC9301E0000E
:10035000130200009B00F0009390C0019380F0FF17
:100360001B01F0001311C101130000001300000075
:1003700063F020201302120093022000E31C52FCC1
:100380009301F000130200009B00F0009390C00165
:100390009380F0FF130000001B01F0001311C10156
:1003A00063F8201C1302120093022000E31E52FC8B
:1003B00093010001130200009B00F0009390C00124
:1003C0009380F0FF130000001B01F0001311C10126
:1003D0001300000063FE2018130212009302200095
:1003E000E31C52FC93011001130200009B00F0007B
:1003F0009390C0019380F0FF1300000013000000F1
:100400001B01F0001311C10163F420161302120046
:1004100093022000E31C52FC930120011302000010
:100420009B00F0009390C0019380F0FF1B01F0004F
:100430001311C10163FE2012130212009302200067
:10044000E31052FE93013001130200009B00F00004
:100450009390C0019380F0FF1B01F0001311C101C4
:100460001300000063F62010130212009302200014
:10047000E31E52FC93014001130200009B00F000B8
:100480009390C0019380F0FF1B01F0001311C10194
:10049000130000001300000063FC200C1302120084
:1004A00093022000E31C52FC930150011302000050
:1004B0009B00F0009390C0019380F0FF13000000B8
:1004C0001B01F0001311C10163F4200A1302120092
:1004D00093022000E31E52FC93016001130200000E
:1004E0009B00F0009390C0019380F0FF1300000088
:1004F0001B01F0001311C1011300000063FA200674
:100500001302120093022000E31C52FC93017001BD
:10051000130200009B00F0009390C0019380F0FF55
:1005200013000000130000001B01F0001311C101B3
:1005300063F020041302120093022000E31C52FC1B
:100540009300100063FA0000938010009380100065
:10055000938010009380100093801000938010000F
:1005600093033000930180016394700063103002A4
:100570000F00F00F638001009391110093E11100CF
:100580009308D00513850100730000000F00F00FE1
:10059000930110009308D0051305000073000000BC
:1005A000731000C000000000000000000000000008
:0C05B0000000000000000000000000003F
:1010000000000000000000000000000000000000E0
:1010100000000000000000000000000000000000D0
:1010200000000000000000000000000000000000C0
:1010300000000000000000000000000000000000B0
:081040000000000000000000A8
:040000058000000077
:00000001FF
